:0600000002005B02379BC9
:03000B000233D8E5
:030013000233E1D4
:03001B0002002BB5
:0300230002364F53
:10002B0032416C636F726E204D634272696465205E
:10003B00496E632E20536372697074204F53202DC9
:10004B002056657273696F6E20362E353320202053
:10005B00C2AF75D0007581567A00122E3D122E4616
:10006B0075B81075A81375B0CF787FE4F6D8FD7509
:10007B008DFD758BFD758C88758A08758921758842
:10008B00047536887535087598C07E007F409020C2
:10009B00007400F0A3DEFCDFFA75A0887800E2F5AF
:1000AB002C75A0887802E2F52DD2AFD28CD28E12AD
:1000BB002158900000123397FAA3123397FBA31227
:1000CB003397FCA3123397FD4C6018A3123397F5AB
:1000DB0040A3123397A3123397F54E9000021221CF
:1000EB00306017903AEA122DB77537287455F59989
:1000FB00780000D8FDD20302019874AAF599780014
:10010B0000D8FDC203903AFB122DB7122D7575382E
:10011B002890000F123397A2E792091231A675456A
:10012B0020754400754B00754A30854E4FE54E6087
:10013B0056900020A3A3D54FFB75A02E7800854EBB
:10014B004F123397F2A308123397F2A308B80002A9
:10015B0005A0D54FEC854E4F854582854483121300
:10016B00A8A3A3123397540F854B82854A83F0A320
:10017B0085824B85834A854582854483A3A38582EB
:10018B0045858344D54FD112324912314C7A001236
:10019B002E3D122E46D29C1201C412021B3001F7C7
:1001AB00C2012003F2123072120C33120F761211AD
:1001BB000D1213CA1213D580DE75D0089021007F63
:1001CB003E7E11E0F5F0A3E0F8A3E0F9686034E5BA
:1001DB00F0547FB400051202558028B401051204B7
:1001EB00ED8020B402051202B28018B40505120A84
:1001FB00818010B40905120B808008B40805120524
:10020B00818000E5822406F5820FDEB775D00022CF
:10021B00300736E4B530130530122D75903B5C1268
:10022B002DB7903B85122DC9801F7405B530100575
:10023B0030903BAE122DB7903BD7122DC9800A746C
:10024B005FB530050530122D9522AC83AD828F83BF
:10025B00898275D00075A0247800E0FB75F000E46E
:10026B0025F0F5F00582E5826508602DE0F208DBEC
:10027B00EF0582C5F003547FB5F01E8582099024EB
:10028B0000E0FBA3D20A753803121420300B0312C3
:10029B00307275D0088982800675373C75D008E5B9
:1002AB00828C838D82F02285820C85830DE50FC3B2
:1002BB00943E23245BF50B850F83850982E030E7A1
:1002CB000FB4F8005007850B82758325F00204D319
:1002DB00850B82758325E0B49000400EB4A00040DE
:1002EB0053B4F00302038B0204D3540FB540F8E56B
:1002FB000904B508030204E6850F83F582E030E7B5
:10030B00030204D31582E00509C3943CB4100050DA
:10031B0020902400F5F0E540F0A37403F0A3E5F082
:10032B00F075D0007BFF902400D20A12142075D0F8
:10033B00080204D3540FB540AEE50904B508030217
:10034B0004E6850F83F582E030E7030204D360B443
:10035B001582E00509C3943CB41000502090240092
:10036B00F5F0E540F0A37402F0A3E5F0F075D000D2
:10037B007BFF902400D20A12142075D0080204D3FC
:10038B00E508C39509B4070050030204BA850F832F
:10039B00850982E0B47F4A0582E0B47F028003B511
:1003AB00403F0582E0B402390582E0B47F02800849
:1003BB00B410028003B430290582E0B407030204B1
:1003CB0072B4010DE508C39509B409005069020424
:1003DB00BAB4060DE508C39509B40A005006020429
:1003EB00BA0204A50582E020E7F760F5B4210050BE
:1003FB00F0F50B0582E020E7E80582E020E7E2F567
:10040B00F00582E020E7DA03548045F0F5F08582B1
:10041B0009902400E540F0A37428F0A3E50B14F039
:10042B00A3E5F0F075D0007BFF902400D20A1214E4
:10043B002075D0080204D30582E020E75DC3943019
:10044B0075F00AA4F5F00582E020E74EC394302541
:10045B00F075F00AA4F5F00582E020E73DC3943077
:10046B0025F014F5F080090582E020E72DC3F5F0A7
:10047B000582E0B4F724858209902400E540F0A3BF
:10048B007418F0A3E5F0F075D0007BFF902400D238
:10049B000A12142075D0080204D330E7030204CEED
:1004AB0075373C850B8275832574F7F00204D38571
:1004BB000F83850982E020E70A0582E582B508F5FE
:1004CB000204E68582091509850C82850D83E509F1
:1004DB0004F0F509650860030202C2850C82850DE4
:1004EB008322AC83AD8275D010E508B509030205F4
:1004FB0076850F83850982E00509B4F5ECA809150B
:10050B0009E508C398B405005003020576120A2AC0
:10051B00B54045902400F0A3F5F0120A2AFBB40372
:10052B0000503525F0F5F0120A2A602CB44000502B
:10053B0027F925F0F5F0E92405FAE508C39509FE3E
:10054B00B512004026120A2AF0A325F0F5F0D9F5D2
:10055B00120A2AB5F002800875373C05090204F42B
:10056B00753803120A3A88090204F475D008E509B4
:10057B008C838D82F022AC83AD8275D010E508B5EB
:10058B00090302064A850F83850982E0B4F10280D4
:10059B0004050980E88509F005F0E508B5F0087554
:1005AB00D0088C838D8222850F8385F082E0B4F195
:1005BB000280DEB4F202800405F080DEE508B509A6
:1005CB000302064A850F83850982E00509B4F10F02
:1005DB0074011209E075A02078C8E4F20205C7B4D3
:1005EB00F216120A0730E00AC2E0C2E11209E00279
:1005FB00065575373C0205C7F5F0120A0720E006D1
:10060B0075373C0205C7F8E5F0B4F009E8D2E11202
:10061B0009E00205C7E830E10BC2E11209E0E5F0A1
:10062B0024F0F5F075A02078C8E275A03378002887
:10063B00F8E5F0F2E80475A02078C8F20205C7755A
:10064B00D008E5098C838D82F02275A02078C8E252
:10065B00B40300500675373C0206F375A0337800DF
:10066B0028F818E2F5F0790018E229F918B8FFF923
:10067B00E9B5F002800675373C0206F375A03378B6
:10068B00009020C412098B120920B4000675373C68
:10069B000206F3B40121E49020B4F0A3F0A3F0A37D
:1006AB00F09020B8F0A3F0A3F0A3F09020BCF0A33F
:1006BB00F0A3F0A3F080129020B412098B9020B815
:1006CB0012098B9020BC12098B7900C0129020C8A4
:1006DB00E0FA1AE4F5F0E2F3080905F0EAB510F6D2
:1006EB00E5F0F0D0120206F602064A120920B40217
:1006FB00399020B4E0B4FF1AA3E0B4FF15A3E0B423
:10070B00FF10A3E0B4FF0B120A07D2E31209E002B9
:10071B0007357582B4E0700FA3E0700BA3E0700790
:10072B00A3E0B5400280030207FE75A0337800906A
:10073B0020C012098B9020C0E0A3B40016E0A3B434
:10074B000011E0A3B4000CE0B404028009B4003B38
:10075B000207FB0207FBE2B4003108E22403FEE2CE
:10076B00FE08902400E540F0A3E2F008A3EEB510DC
:10077B00F890240075D000D20A7538031214207536
:10078B00D010120A0730E3090207FE75373C020747
:10079B00FB75A02078C4120948120920B402147505
:1007AB00A02078B812094875A02078B412094874B3
:1007BB0005F0A3E4F0A37401F0A375A02078C8E2C0
:1007CB00F975A0337800E2F008A3E8B511F875A02D
:1007DB0024780075F000A982E20825F0F5F0E8B561
:1007EB0011F6E5F0F0A3E50FC3943EFA091208BE2B
:1007FB000208679020BCE0700EA3E0700AA3E070C3
:10080B0006A3E07002805514F0B4FF187582BEE0A9
:10081B0014F0B4FF0F7582BDE014F0B4FF067582BF
:10082B00BCE014F0E50FC3943EF5F0902100E58297
:10083B002408F5827A01E0547FB40816E5F0B5126E
:10084B0002800FAD82AE83AFF012086A8D828E8369
:10085B008FF0E5822408F5820ABA11DA0206F390CA
:10086B00240075A02078C412094875A02078B41212
:10087B00094875A02078B812094875A02078BC12D9
:10088B00094875A02078C8E2F975A0337800E2F02A
:10089B0008A3E8B511F875A024780075F000A982BB
:1008AB00E20825F0F5F0E8B511F6E5F0F0A3091232
:1008BB0008BE2290340074F1F0A375A0247800E2F6
:1008CB0008B4F007F0A3E4F0A3801CB4F10A74F0B1
:1008DB00F0A37401F0A3800FB4F20A74F0F0A374C8
:1008EB0002F0A38002F0A3E8B511D474F2F0A3A92F
:1008FB008290240075A0347800E2F008A3E582B55D
:10090B0011F775D000902400AB11AA12D20A122E47
:10091B004F75D01022C082C0839020C4E0B4001663
:10092B00A3E0B40011A3E0B4000CA3E0B401028077
:10093B0007B4020280027400D083D08222E20860E6
:10094B001674FDF0A30808E218F0A3E218F0A3E276
:10095B0018F0A3E2F0A322E208601174FEF0A308E2
:10096B00E218F0A3E218F0A3E2F0A322E208600C75
:10097B0074FFF0A3E218F0A3E2F0A322E2F0A322AB
:10098B00C011E2F9B9FD1708080808E218F0A3E254
:10099B0018F0A3E218F0A3E2F00808088033B9FEC0
:1009AB0014E4F0A3080808E218F0A3E218F0A3E29D
:1009BB00F00808801CB9FF10E4F0A3F0A30808E2CC
:1009CB0018F0A3E2F0088009E4F0A3F0A3F0A3E28F
:1009DB00F008D01122C009C082C083C0E0E50FC36C
:1009EB00943EF509902100E5822408D509FB2407E4
:1009FB00F582D0E0F0D083D082D00922C009C0822A
:100A0B00C083E50FC3943EF509902100E5822408CD
:100A1B00D509FB2407F582E0D083D082D00922C010
:100A2B0083C082850F838882E008D082D0832275B1
:100A3B00D0007BFF902400D20A121420E513B400DF
:100A4B0002802FB40214E50FC3943EFA850F838501
:100A5B000982E516FBD20A122E4FE50FC3943EFA1C
:100A6B0074AA3012027455902400F07B01D20A1242
:100A7B002E4F75D01022AC83AD8275D010A809E52E
:100A8B0008C398B40C005003020B75850F83E5095E
:100A9B002402F582E0B43A028066B42D60A809E521
:100AAB0008C398B417005003020B75E5092416F51B
:100ABB0082E0B40D48902400A8097919120BD612C4
:100ACB000C0608791A120BD6120C0608791B120B9E
:100ADB00D6120C06E82406F8791C120BD6120C065B
:100AEB0008791D120BD6120C0608791E120BD612A2
:100AFB000C06791FE4120C06E8F5098080020B70D6
:100B0B00E509240BF582E0B40D5BA809E8F9120B9B
:100B1B00D6B41800504C120A2AB43A46120BD6B46B
:100B2B003C00503E120A2AB43A38120BD6B43C00A1
:100B3B005030753803902400E9F8791C120BD6124B
:100B4B000C0608791D120BD6120C0608791E120B17
:100B5B00D6120C06791FE4120C06E509240CF509D4
:100B6B00418875373C0509020A8875D008E5098C60
:100B7B00838D82F022AC83AD8275D010A809E50875
:100B8B00C398B405004039850F83850982E0B443CF
:100B9B002AA809E5092403F8E8120BD6601AB463F6
:100BAB0000501514758330F582E0D2E2F0753803EE
:100BBB00E5092405F50980C475373C0509020B8747
:100BCB0075D008E5098C838D82F022C083C08285A5
:100BDB000F838882E0080582C39430B4060050145A
:100BEB0075F00AA4F5F0E008C39430B40A00500481
:100BFB0025F0800274FFD082D08322C0F0F5F0E59F
:100C0B0040F0A37428F0A3E9F0A3E5F0F0A32428A7
:100C1B002903547FF075D0007BFF902400D20A1279
:100C2B00142075D010D0F022908800E0F8C52C6805
:100C3B0030E00CC0E0A26075F000120D2CD0E0305B
:100C4B00E10CC0E0A26175F001120D2CD0E030E296
:100C5B000CC0E0A26275F002120D2CD0E030E30C58
:100C6B00C0E0A26375F003120D2CD0E030E40CC091
:100C7B00E0A26475F004120D2CD0E030E50CC0E05E
:100C8B00A26575F005120D2CD0E030E60CC0E0A289
:100C9B006675F006120D2CD0E030E708A26775F0F0
:100CAB0007120D2C908802E0F8C52D6830E00CC0BF
:100CBB00E0A26875F008120D2CD0E030E10CC0E01A
:100CCB00A26975F009120D2CD0E030E20CC0E0A245
:100CDB006A75F00A120D2CD0E030E30CC0E0A26B69
:100CEB0075F00B120D2CD0E030E40CC0E0A26C754B
:100CFB00F00C120D2CD0E030E50CC0E0A26D75F0BD
:100D0B000D120D2CD0E030E60CC0E0A26E75F00E8B
:100D1B00120D2CD0E030E708A26F75F00F120D2CDE
:100D2B0022920590257DE07003020E8EF54F754DD6
:100D3B0000754C26854D82854C83E0F9A3E0FAA320
:100D4B00E0A3A385824D85834C89828A83F545C0B8
:100D5B00F075F002A4F54B85F04AD0F0A3A3123343
:100D6B0097FBA3123397FCA3123397FDA312339770
:100D7B00FEA3123397FFEF547FB5F05EEB20E40533
:100D8B002005578003300552EE600CB40700500766
:100D9B00120E9240028043903000E5452582F58289
:100DAB00E030E23030E02FE54B2400F582E54A34A9
:100DBB0031F5831213BBE582C39CE5839D5003027F
:100DCB000E8BE545121E84758330854582E0D2E299
:100DDB00F0020E8BD2E2F0020E8BA3123397FEA31E
:100DEB00123397FFEF547FB5F02BEB20E505200571
:100DFB0024800330051FEE600CB407005007120E61
:100E0B009240028010903000E5452582F582E0C2C9
:100E1B00E2F0020E8BA3123397FEA3123397FFEF70
:100E2B00547FB5F02BEB20E605200524800330051D
:100E3B001FEE600CB407005007120E924002801098
:100E4B00903000E5452582F582E0D2E3F0020E8B6F
:100E5B00A3123397FEA3123397FFEF547FB5F02005
:100E6B00EB20E7052005198003300514EE600CB468
:100E7B0007005007120E9240028005E545121E84B2
:100E8B00D54F0122020D3FC082C083C0F0E5822402
:100E9B0007F582E5833400F583123397F8A31233F9
:100EAB0097541F240BF975A025E3F9EE30E708E8FA
:100EBB00541F240BF8E2F8EE540F2323900ECB7340
:100ECB00020F0B00020F0F00020F1D00020F2B0071
:100EDB00020F3B00020F4D00020F5D00020F0F00CF
:100EEB00020F1D00020F2B00020F3B00020F4D00E3
:100EFB00020F5D00020F0B00020F0B00020F0B0025
:100F0B00C3020F6FE988F0B5F004D3020F6FC30271
:100F1B000F6FE988F0B5F004C3020F6FD3020F6FA8
:100F2B00E988F0B5F0004004C3020F6FD3020F6FD6
:100F3B00E988F0B5F00280064004C3020F6FD302BC
:100F4B000F6FE889F0B5F00040E2C3020F6FD302D8
:100F5B000F6FE889F0B5F00280064004C3020F6FF3
:100F6B00D3020F6FD0F0D083D08222200F03021058
:100F7B00A590257EE070030210A5F54F754D007509
:100F8B004C2A854D82854C83E0F9A3E0FAA3E0A3BC
:100F9B00A385824D85834C89828A83F545C0F07584
:100FAB00F002A4F54B85F04AD0F0A3A3123397FBC4
:100FBB00A3123397FCA3123397FDA3123397FEA30F
:100FCB00123397FFEE541FB40700404A1210A8408B
:100FDB00028043903000E5452582F582E030E23017
:100FEB0030E02FE54B2400F582E54A3431F58312CE
:100FFB0013BBE582C39CE5839D5003021091E5452D
:10100B00121E84758330854582E0D2E2F002109186
:10101B00D2E2F0021091A3123397FEA3123397FF83
:10102B00EE541FB4070040171210A8400280109016
:10103B003000E5452582F582E0C2E2F0021091A373
:10104B00123397FEA3123397FFEE541FB4070040E1
:10105B00171210A840028010903000E5452582F54C
:10106B0082E0D2E3F0021091A3123397FEA3123366
:10107B0097FFEE541FB40700400C1210A8400280DB
:10108B0005E545121E84D54F0302109A020F8D7E83
:10109B002090252B7400F0A3DEFCC20F22C082C06F
:1010AB0083C0F0E5822407F582E5833400F58312D3
:1010BB003397F8A3123397541FF990252B2582F5FC
:1010CB0082E0C2046002D204EE30E719E8541FF844
:1010DB0090252B2582F582E06002D20475A0257441
:1010EB000B28F8E2F830041275A025740B29F9E3EC
:1010FB00F9EE540F2323900ECB73C3D0F0D083D0D3
:10110B008222854E4FE54E7003021366754B0075B8
:10111B004A30754D00754C2E900020E54E12136D24
:10112B008582478583467543007542317545207529
:10113B004400854B82854A83E020E2030212FC9037
:10114B00001C1233975401700890001B12339760E8
:10115B00328545828544831213A874152582F58246
:10116B0074003583F58312339730E017C082C08348
:10117B0020E104740080027401903504F0D083D018
:10118B00828011C082C0837400903504F0D083D06C
:10119B0082021275A3123397F8A3123397F9A31295
:1011AB003397FA903502E0FB903501E0FC90350067
:1011BB00E0FDC3EB98F582EC99F5838542A0A8433B
:1011CB00E582F208E583F2ED9A30E70302126370D1
:1011DB0071903505854FF0C3E58225F0F582E583E7
:1011EB003400F583E020E211E2701718E275F00588
:1011FB00B5F002800440028009903503E0700302D1
:10120B00128B903504E070030212BC854782854631
:10121B00831213A88582498583481213A8E582455A
:10122B0083601F121380600A854982854883A3A3BC
:10123B0080E2854D82854C83E549F0A3E548F002B9
:10124B0012EF903504E06069854D82854C83E5494A
:10125B00F0A3E548F00212EF85478285468312130F
:10126B00A88582498583480212EF85438285428394
:10127B001213BBA38542A0A843E582F208E583F2D3
:10128B00854D82854C831213BB8582498583481219
:10129B0013A8E582458360191213806047A3A3C28C
:1012AB000A12142020063D854982854883A3A3801A
:1012BB00D8903504E0702D8547828546831213A89C
:1012CB008582498583488542A0A8437400F208F2C1
:1012DB00854B82854A83E030E10510E3028002C230
:1012EB00E2C2E4F0854D82854C83E549F0A3E548E5
:1012FB00F0854B82854A83E0F9903505854FF0C325
:10130B00E58225F0F582E5833400F583E9F0D54FCE
:10131B00028048854B82854A83A385824B85834A0D
:10132B00854D82854C83A3A385824D85834C854750
:10133B0082854683A3A38582478583468543828521
:10134B004283A3A38582438583428545828544835B
:10135B00A3A385824585834402113D903503740018
:10136B00F022C0F075F002A42582F582E5F03583FA
:10137B00F583D0F022AD82AE831213A8AB82AC837F
:10138B008543828542831213BBE582C39BE5839C15
:10139B00400474FF800274008D828E8322C0F01291
:1013AB003397F5F0A3123397F58385F082D0F022B3
:1013BB00C0F0E0F5F0A3E0F58385F082D0F022AA2F
:1013CB0024122E3DAA25122E4622301347E550B487
:1013DB00024214F550780075A02574FFF208E54021
:1013EB00F2087400F208E52CF208E52DF208E52E60
:1013FB00F208E52FF208908000E0F208A3A3E0F2D8
:10140B0008A3A3E0F208E4F208F29025007A007B2F
:10141B002B122E4F22C206AD82AE837A001233B24C
:10142B00FFA31233B2C212B467004003D212229050
:10143B0039EC75F002A42582F582E5F03583F5834E
:10144B00E493F5F0A3E49385F083F582E47312162D
:10145B000502160012164702160012168802160015
:10146B001216C802160012170E021600121750029F
:10147B00160012175F02160012179E0216001217A3
:10148B00B60216001217CE0216001217F70216003C
:10149B0012194E0216001231140216001219AC0268
:1014AB0016001219F3021600121B16021600121C5C
:1014BB0039021600121C70021600121CC302160011
:1014CB00121D16021600121D77021600121C4E0278
:1014DB001600121DD8021600121E3E021600121E16
:1014EB0057021600121E70021600121FA5021600DC
:1014FB001220B60216001222DE021600021600128D
:10150B002D75021600122D950216001223340216A9
:10151B000012236202160012240C02160012243051
:10152B0002160012245C0216001224890216001205
:10153B0024BA0216001224E902160012251C021608
:10154B000012254D0216001225870216001225C225
:10155B0002160012260102160012263E0216001277
:10156B00267F0216001226BE0216001226E5021670
:10157B000012270E02160012273A02160012276BD2
:10158B0002160012279E0216001227D50216001211
:10159B00280A02160012284302160012287A021695
:1015AB00001228B90216001228FA02160012293F5F
:1015BB000216001229820216001229C90216001205
:1015CB002A0E021600122A3D021600122390021652
:1015DB00001223C6021600122A6E021600122AF7F8
:1015EB00021600122B2D021600122D5F021600128E
:1015FB002B6C0216008D828E83228D828E83A3A389
:10160B001233B220E629122116B900104224F4F548
:10161B00F0902040E055F0F05228801FB9011042A5
:10162B0025F4F5F0902041E055F0F05229800C5450
:10163B003F2474F58275832074FFF0228D828E8394
:10164B00A3A31233B220E628122116F4B9000F52CD
:10165B0024F5F0902040E055F0F05228801EB9019F
:10166B000F5225F5F0902041E055F0F05229800CF7
:10167B00543F2474F5827583207400F0228D828E82
:10168B0083A3A31233B2F8541F232400C8122116CC
:10169B00FAA31233B275A020F208F2EAB9000DF5E5
:1016AB00F0902040E045F0F042288010B9010DF594
:1016BB00F0902041E045F0F042298000228D828E8F
:1016CB0083A3A31233B2F8541F232400C81221168C
:1016DB00FAA31233B275A020F208F2EAB900104255
:1016EB00286224F4F5F0902040E055F0F08013B917
:1016FB00011042296225F4F5F0902041E055F0F0FD
:10170B008000228D828E83A3A31233B220E629128E
:10171B002116B900106224F4F5F0902040E055F04A
:10172B00F05228801FB901106225F4F5F09020418A
:10173B00E055F0F05229800C543F2474F5827583E8
:10174B0020E0F4F0228D828E83A3A31233B2FBA38D
:10175B001221B622902200E0F8A3E0F5F075A04F1D
:10176B00902100E0547FB40105790102177B7900C9
:10177B00903ABCE993600BF20908E8B5F0F5D20694
:10178B008010902200E8C2ACF0200804D208D29955
:10179B00D2AC228D828E83A3A31233B2FAA312335F
:1017AB00B2FBA3122E4F6002D206228D828E83A330
:1017BB00A31233B2FAA31233B2FBA3122ECA6002E6
:1017CB00D206228D828E83A3A31233B2FA7B01A39E
:1017DB001233B290250B2582F582A20AC0D0D20A11
:1017EB00122E4FD0D0920A6002D206228D828E83A7
:1017FB00A3A31233B2FAA31233B2C0E0A31233B2D3
:10180B00FF54072323901814730218330002186532
:10181B0000021890000218B50002183300021833AA
:10182B000002183300021833D0E090250B2582F507
:10183B0082E0780079007C00600F75F00A84A8F0D4
:10184B00600775F00A84A9F0FCE82430F8E924302D
:10185B00F9EC2430FC7B030218D3D0E090250B2548
:10186B0082F582E0540F2430B43A0040022407F989
:10187B00E054F0C42430B43A0040022407FC782032
:10188B007B020218D3D0E090250B2582F582E05421
:10189B00072430F8E054380303032430F9E054C034
:1018AB0023232430FC7B030218D3D0E090250B2597
:1018BB0082F5827B01A20AC0D0D20A122E4FD0D061
:1018CB00920A607ED206807AEF5438039018DB734D
:1018DB000218FA0002192E0002191F000219080043
:1018EB000218FA000218FA000218FA000218FABBE2
:1018FB000102802FBC302CE9FCE8F9DBF2BC302371
:10190B00E9FCE8F97820BB031ABC3017E9FCE8F9CD
:10191B007820800FBC300C7C20BB0307B9300479D6
:10192B00208000902044ECF0A3E9F0A3E8F0902095
:10193B0044A20AC0D0D20A122E4FD0D0920A600213
:10194B00D206228D828E83A3A31233B2FAA3123353
:10195B00B2F8A31233B2F9A31233B290250B25823E
:10196B00F582E0FB9020447406F0A3E5404480F040
:10197B00FCA3E8F02CFCA37428F02CFCA3E9F02CBE
:10198B00FCA3EBF02CA303547FF09020447B07A225
:10199B000AC0D0D20A122E4FD0D0920A6002D206C1
:1019AB00228D828E8375D010A3A31233B2FBA3AD0D
:1019BB0082AE83902100E5822408F5827A01E054FF
:1019CB007FB40819A882A9838D828E8375D000AA53
:1019DB0012AB13122E4F75D01088828983E58224A7
:1019EB0008F5820ABA11D722854B82854A83E0F922
:1019FB008D828E83A3A31233B2FA232323FC75A00B
:101A0B0021F8E920E442E2C2E7F2E408F208F2A38B
:101A1B001233B2FBA3122E4F75A021ECF8E2D2E7E2
:101A2B00F208080808081233B2F2A3081233B2F214
:101A3B00200606A3081233B2F2854B82854A83E057
:101A4B00D2E4F0D206021B1508A31233B2240525EB
:101A5B0082F582E43583F5831233B2F5F0E2C39558
:101A6B00F0501E08080808E2F5F008E245F0602D7A
:101A7B0018E2C39401F2500408E214F2D206021BDE
:101A8B0015ABF0A3EA243EF5A078001233B2F5F0C3
:101A9B00E2B5F009A308DBF3753803804A75A02182
:101AAB00EC2407F8E2600F14F28D828E83A3A3EC73
:101ABB00F8D206021A1175373C30092B900014121C
:101ACB003397F8A3123397F5838882E5822AF58240
:101ADB00E43583F583123397F8C3954E500975831C
:101AEB00308882E0D2E2F075A021ECF8E2547FB4AA
:101AFB0003028003B40704C2E78002D2E7F2854BEE
:101B0B0082854A83E0C2E4F0C20622854B82854A75
:101B1B0083E0F98D828E83A3A31233B2FA2323239E
:101B2B00FC75A021F8E920E442E2C2E7F2E408F2F6
:101B3B0008F2A31233B2FBA3122ECA75A021ECF844
:101B4B00E2D2E7F208080808081233B2F2A308122F
:101B5B0033B2F2200606A3081233B2F2854B82850C
:101B6B004A83E0D2E4F0D206021C3808A31233B247
:101B7B0024052582F582E43583F5831233B2F5F023
:101B8B00E2C395F0501E08080808E2F5F008E2459C
:101B9B00F0602D18E2C39401F2500408E214F2D263
:101BAB0006021C38ABF0A3EA243EF5A078001233F2
:101BBB00B2F5F0E2B5F009A308DBF3753803804A00
:101BCB0075A021EC2407F8E2600F14F28D828E834E
:101BDB00A3A3ECF8D206021B3475373C30092B90CB
:101BEB000014123397F8A3123397F5838882E5829A
:101BFB002AF582E43583F583123397F8C3954E505B
:101C0B00097583308882E0D2E2F075A021ECF8E20E
:101C1B00547FB403028003B40704C2E78002D2E707
:101C2B00F2854B82854A83E0C2E4F0C206228D82A4
:101C3B008E83A3A31233B2547F232549F549500257
:101C4B000548228D828E83A3A31233B2FAA31233DB
:101C5B00B2F9EAC333FAE933F9EAC32549F549E99D
:101C6B003548F548228D828E83A3A31233B220E729
:101C7B001F10E611122116B9000478248025B90132
:101C8B00047825801E2474F875A020E2701A802732
:101C9B00547F122116B90004782C8007B9010478FF
:101CAB002D8000567002800FA31233B2547F232570
:101CBB0049F54950020548228D828E83A3A3123326
:101CCB00B220E71F10E611122116B9000478248008
:101CDB0025B901047825801E2474F875A020E260D4
:101CEB001A8027547F122116B90004782C8007B96B
:101CFB000104782D8000566002800FA31233B2547A
:101D0B007F232549F54950020548228D828E83A3F6
:101D1B00A31233B220E71F10E611122116B90004EB
:101D2B0078248025B901047825801E2474F875A0C9
:101D3B0020E2701A8035547F122116B90004782CDA
:101D4B008007B90104782D8000567002801DA31204
:101D5B0033B2FAA31233B2F9EAC333FAE933F9EA2D
:101D6B00C32549F549E9FA3548F548228D828E831A
:101D7B00A3A31233B220E71F10E611122116B900EC
:101D8B000478248025B901047825801E2474F87505
:101D9B00A020E2601A8035547F122116B900047816
:101DAB002C8007B90104782D8000566002801DA39A
:101DBB001233B2FAA31233B2F9EAC333FAE933F9A5
:101DCB00EAC32549F549E9FA3548F548228D828E53
:101DDB0083A3A31233B2F8C3954E50567583308844
:101DEB0082E030E24A30E04AC004C005900020E8AF
:101DFB0012136D1213A8A3A3A3123397FCA31233D0
:101E0B0097FDE8C0F075F002A42400F582E5F034EC
:101E1B0031F583D0F01213BBE582C39CE5839DD0D3
:101E2B0005D004400DE8121E847583308882E0D201
:101E3B00E2F0228D828E83A3A31233B2F8C3954EA8
:101E4B0050097583308882E0C2E2F0228D828E8346
:101E5B00A3A31233B2F8C3954E5009758330888211
:101E6B00E0D2E3F0228D828E83A3A31233B2F8C3A8
:101E7B00954E5004E8121E8422C000C003C004C05B
:101E8B00F0F8900020E54E12136DE812136D12134B
:101E9B00A8AB82AC8375832EE875F002A4F582E5BE
:101EAB00F03583F583EBF0A3ECF0758331E875F037
:101EBB0002A4F582E5F03583F583E4F0A3F0758396
:101ECB00308882E0C2E2C2E4F0C2E3D0F0D004D0AA
:101EDB0003D00022902200E0F875A04F902100E083
:101EEB00547FB400047402F208900002123397A3DB
:101EFB00F208123397F208902200E8C2ACF02008E7
:101F0B0004D208D299D2AC22C004C005C00675A079
:101F1B0025784B791075040075050075060CD504F2
:101F2B001DD5051AD506177455C29BC299F599751F
:101F3B000400750504D504FDD505FA02005B309845
:101F4B00DDE599F2C298EA70011B1AEB7003EA60A7
:101F5B001108D9C1784B7910E212337AA308D9F85A
:101F6B0080AC7A007B20DAFEDBFC784B7910E21236
:101F7B00337AA308D9F8902100E0547FB40114748C
:101F8B00AAC29BC299F599750400750508D504FD85
:101F9B00D505FAD006D005D00422C2AF8D828E8330
:101FAB00A3A31233B2FAA31233B2FBE599C298740E
:101FBB00AAC29BC299F599900000121F1302005BF5
:101FCB008D828E83A3A31233B2FAA31233B2FB908A
:101FDB000002123397F8A3123397C854F0241CC88D
:101FEB00500104F5838882745A12337AA374A512B4
:101FFB00337AA3EA12337AA3EB12337AA3C000C06D
:10200B0001750000750100D500FDD501FAD001D096
:10201B0000C2AFE599C29874AAC29BC299F59912F6
:10202B001F1374AAC29BC299F59975040075050418
:10203B00D504FDD505FA02005B2014FDC29BD2141A
:10204B00F59922900002123397F8A3123397C854D4
:10205B00F0241CC8500104F5838882123397B45ABC
:10206B0018A3123397B4A511A3123397FAA3123303
:10207B0097FBA3BA000CBB0009E4122044122044C6
:10208B00801AEA122044EB122044123397A3122039
:10209B00441ABAFF011BBA00F1BB00EE75040075C0
:1020AB000504D504FDD505FA02005B90000212333E
:1020BB0097FAA3123397FB700CEA7009E4122044D1
:1020CB0012204480278A828B83A3A3AA82AB83EA44
:1020DB00122044EB122044900000123397A31220DD
:1020EB00441ABAFF011BBA00F1BB00EE7504007570
:1020FB000504D504FDD505FA02005B8D828E83A302
:10210B00A31233B2C2136002D21322F95407C903CC
:10211B0003035403C0E07401B90002800323D9FD0B
:10212B00F9D0E0C9227800790012339728500109C1
:10213B00F8A3DC05BD00F28006BCFFED1D80EAE8CC
:10214B006A7007E96B7003E4800274FF2290000051
:10215B0075A0987802E230E70BA3E583B405F6C2CD
:10216B00110221B5D2117A30122DDB7A30122DDB10
:10217B007A38122DDB7A80122DDB7A06122DDB7A60
:10218B000C122DDB7A01122DDB7A40122DDB7A5AE1
:10219B00122DFA7A40122DDB122E1CB45AC1903A32
:1021AB00D9122DB7903AC8122DC922EB60627A80F2
:1021BB00122DDB1233B2B404005029A3DB02805082
:1021CB00B400047A808010B401047AC08009B40290
:1021DB00047A9480027AD41233B2A3543F2AFA12AF
:1021EB002DDB802AB40C08A37A01122DDB801FB4DF
:1021FB000D03A38014B40A03A3800EB40E2EDB11BF
:10220B00800EFA122DFAA380057AC0122DDBDBA308
:10221B0022A31233B214A3C082C08390250B258254
:10222B00F582E0D083D08212229A80E2B40FD3DB06
:10223B000280DDA31233B214A3C082C08390250B9E
:10224B002582F582E0D083D08212225980C07C0196
:10225B007A20C39464400C1C7A31C394644004C349
:10226B0094640A2464C0E0122DFAD0E07A31C3944E
:10227B000A40030A80F81A240AC0E0BA3005EC6061
:10228B00027A20122DFAD0E02430FA122DFA227C99
:10229B00017A20C39464400C1C7A31C394644004CB
:1022AB00C394640A2464BA20028007C0E0122DFA9A
:1022BB00D0E07A31C3940A40030A80F81A240AC08A
:1022CB00E0BA3003EC7003122DFAD0E02430FA128E
:1022DB002DFA228D828E83A3A31233B25403FB708B
:1022EB0005903B0C8013B40105903B1C800BB40292
:1022FB0005903B2C8003903B3C7A01122DDB7C102C
:10230B00E493FA122DFAA3DCF77C107AC0122DDBC2
:10231B00EBC42474F582758320E060047A3180026B
:10232B007A30122DFAA3DCF1228D828E83A3A312B5
:10233B0033B2FAA31233B2FBEA4224F4F5F0902045
:10234B0040E055F0F05228EB4225F4F5F090204197
:10235B00E055F0F05229228D828E83A3A31233B263
:10236B00FAA31233B2FBEAF45224F5F0902040E0CA
:10237B0055F0F05228EBF45225F5F0902041E05542
:10238B00F0F05229228D828E83A3A31233B2FAA3CB
:10239B001233B2FBEA7011EBF524F4F5F090204008
:1023AB00E055F0F052288012B4010FEBF525F4F54F
:1023BB00F0902041E055F0F05229228D828E83A3BC
:1023CB00A31233B2FAA31233B2FBEA701875A0252D
:1023DB00740B2BF8E52CF275A025742B2BF874FFDE
:1023EB00F2D20F801BB4011875A025740B2BF8E5E6
:1023FB002DF275A025742B2BF874FFF2D20F8000F1
:10240B00228D828E83A3A31233B2541FF9240BF8AF
:10241B00A31233B275A025F275A025742B29F8747D
:10242B00FFF2D20F228D828E83A3A31233B2541FDD
:10243B00F9240BF875A025E2F5F0A31233B2B5F031
:10244B000FA31233B2547F232549F5495002054897
:10245B00228D828E83A3A31233B2541F240BF875E3
:10246B00A025E2F5F0A31233B2B5F002800FA31250
:10247B0033B2547F232549F54950020548228D82FA
:10248B008E83A3A31233B2541F240BF875A025E23D
:10249B00F5F0A31233B2C5F0B5F0004002800FA3E4
:1024AB001233B2547F232549F54950020548228D3A
:1024BB00828E83A3A31233B2541F240BF875A0256D
:1024CB00E2F5F0A31233B2B5F0004002800FA31275
:1024DB0033B2547F232549F54950020548228D829A
:1024EB008E83A3A31233B2541F240BF875A025E2DD
:1024FB00F5F0A31233B2C5F0B5F0028004400280B0
:10250B000FA31233B2547F232549F54950020548D6
:10251B00228D828E83A3A31233B2541F240BF87522
:10252B00A025E2F5F0A31233B2B5F002800440020D
:10253B00800FA31233B2547F232549F5495002056E
:10254B0048228D828E83A3A31233B2541FF9240B1E
:10255B00F875A025E2F5F0A31233B2B5F01DA31266
:10256B0033B2FAA31233B2F9EAC333FAE933F9EA15
:10257B00C32549F549E9FA3548F548228D828E8302
:10258B00A3A31233B2541F240BF875A025E2F5F068
:10259B00A31233B2B5F002801DA31233B2FAA31209
:1025AB0033B2F9EAC333FAE933F9EAC32549F549FA
:1025BB00E9FA3548F548228D828E83A3A31233B2F4
:1025CB00541F240BF875A025E2F5F0A31233B2C506
:1025DB00F0B5F0004002801DA31233B2FAA3123300
:1025EB00B2F9EAC333FAE933F9EAC32549F549E904
:1025FB00FA3548F548228D828E83A3A31233B25449
:10260B001F240BF875A025E2F5F0A31233B2B5F039
:10261B00004002801DA31233B2FAA31233B2F9EABF
:10262B00C333FAE933F9EAC32549F549E9FA3548E1
:10263B00F548228D828E83A3A31233B2541F240B31
:10264B00F875A025E2F5F0A31233B2C5F0B5F00290
:10265B0080044002801DA31233B2FAA31233B2F9E5
:10266B00EAC333FAE933F9EAC32549F549E9FA35FF
:10267B0048F548228D828E83A3A31233B2541F24B4
:10268B000BF875A025E2F5F0A31233B2B5F002807A
:10269B00044002801DA31233B2FAA31233B2F9EA3B
:1026AB00C333FAE933F9EAC32549F549E9FA354861
:1026BB00F548228D828E83A3A31233B2541FF924C3
:1026CB000BF875A025E2FAA31233B22AF275A025F6
:1026DB00742B29F974FFF3D20F228D828E83A3A35F
:1026EB001233B2541FF9240BF875A025E2FAA3128A
:1026FB0033B2CAC39AF275A025742B29F974FFF370
:10270B00D20F228D828E83A3A31233B2541FF5F006
:10271B00240BF8A31233B2541F240BF975A025E335
:10272B00F275A025742B25F0F874FFF2D20F228DD1
:10273B00828E83A3A31233B2541F240BF875A025EA
:10274B00E2F5F0A31233B2541F240BF9E3B5F00FEB
:10275B00A31233B2547F232549F549500205482271
:10276B008D828E83A3A31233B2541F240BF875A052
:10277B0025E2F5F0A31233B2541F240BF9E3B5F0A5
:10278B000280DCA31233B2547F232549F549500252
:10279B000548228D828E83A3A31233B2541F240BC0
:1027AB00F875A025E2F5F0A31233B2541F240BF9F0
:1027BB00E3C5F0B5F0004002800FA31233B2547F93
:1027CB00232549F54950020548228D828E83A3A308
:1027DB001233B2541F240BF875A025E2F5F0A312A7
:1027EB0033B2541F240BF9E3B5F0004002800FA362
:1027FB001233B2547F232549F54950020548228DE7
:10280B00828E83A3A31233B2541F240BF875A02519
:10281B00E2F5F0A31233B2541F240BF9E3C5F0B564
:10282B00F00280044002800FA31233B2547F2325A1
:10283B0049F54950020548228D828E83A3A312339A
:10284B00B2541F240BF875A025E2F5F0A31233B296
:10285B00541F240BF9E3B5F00280044002800FA350
:10286B001233B2547F232549F54950020548228D76
:10287B00828E83A3A31233B2541F240BF875A025A9
:10288B00E2F5F0A31233B2541F240BF9E3B5F01D9C
:10289B00A31233B2FAA31233B2F9EAC333FAE93310
:1028AB00F9EAC32549F549E9FA3548F548228D82FD
:1028BB008E83A3A31233B2541F240BF875A025E209
:1028CB00F5F0A31233B2541F240BF9E3B5F00280D9
:1028DB00DCA31233B2FAA31233B2F9EAC333FAE927
:1028EB0033F9EAC32549F549E9FA3548F548228D0C
:1028FB00828E83A3A31233B2541F240BF875A02529
:10290B00E2F5F0A31233B2541F240BF9E3C5F0B573
:10291B00F0004002801DA31233B2FAA31233B2F9B6
:10292B00EAC333FAE933F9EAC32549F549E9FA353C
:10293B0048F548228D828E83A3A31233B2541F24F1
:10294B000BF875A025E2F5F0A31233B2541F240B3C
:10295B00F9E3B5F0004002801DA31233B2FAA312C3
:10296B0033B2F9EAC333FAE933F9EAC32549F54936
:10297B00E9FA3548F548228D828E83A3A31233B230
:10298B00541F240BF875A025E2F5F0A31233B254B3
:10299B001F240BF9E3C5F0B5F00280044002801D43
:1029AB00A31233B2FAA31233B2F9EAC333FAE933FF
:1029BB00F9EAC32549F549E9FA3548F548228D82EC
:1029CB008E83A3A31233B2541F240BF875A025E2F8
:1029DB00F5F0A31233B2541F240BF9E3B5F00280C8
:1029EB00044002801DA31233B2FAA31233B2F9EAE8
:1029FB00C333FAE933F9EAC32549F549E9FA35480E
:102A0B00F548228D828E83A3A31233B2541FF5F0A7
:102A1B00240BF875A025E2FAA31233B2541F240B32
:102A2B00F9E32AF275A025742B25F0F874FFF2D286
:102A3B000F228D828E83A3A31233B2541FF5F02481
:102A4B000BF875A025E2FAA31233B2541F240BF92D
:102A5B00E3CAC39AF275A025742B25F0F874FFF224
:102A6B00D20F228D828E83A3A31233B2541FF990FF
:102A7B003B4C7A01122DDB7C10E493FA122DFAA356
:102A8B00DCF77AC0122DDB9024007420F0A3F0A3A6
:102A9B00F0A3F0A3E904122C66EBB430027420F01F
:102AAB00A3EAF0A37420F0A3743DF0A37420F0A369
:102ABB0075A025E9240BF9E3122C66ECD204B43093
:102ACB0004C2047420F0A3EBB4300520040274207C
:102ADB00F0A3EAF0A37420F0A3F0A3F0A3F07C1012
:102AEB00902400E0FA122DFAA3DCF8228D828E835B
:102AFB00A3A31233B2541FF9FB75A025240BF9E3E2
:102B0B00FA90001A123397C39401B408005012C400
:102B1B0023441FF583EB44E0F582EA12337A122D3E
:102B2B006A228D828E83A3A31233B2541FF99000B5
:102B3B001A123397C39401B408005024C423441FC2
:102B4B00F583E944E0F582123397FA75A025740BEF
:102B5B0029F8EAF275A025742B29F874FFF2D20F2D
:102B6B0022C0F08D828E83A3A31233B275F03CA4E6
:102B7B00FEAFF0A31233B2C32EFEEF3400FFA3124D
:102B8B0033B275F03CFB7C007D00C3EB2EFBEC3FBE
:102B9B00FCED3400FD15F0E5F070EFA31233B2F845
:102BAB0079007A00900009123397B4000575F0187C
:102BBB008013B4030575F019800BB4010575F01E75
:102BCB00800375F01EC3E82BF8E93CF9EA3DFA15D2
:102BDB00F0E5F070F0900009123397B4013AEF7002
:102BEB000BEE6034B40A03022BF74018C3EE940AC1
:102BFB00FEEF9400FFC3E89412F8E99400F9EA940D
:102C0B0000FA80DAC3EE9401FEC3E89402F8E9946B
:102C1B0000F9EA9400FA80C6903500E0FD9035018A
:102C2B00E0FC903502E0FBC3E89BFFE99C7014EAE3
:102C3B009D701090001B123397F5F0EFB5F00280EA
:102C4B000840069035037401F0903500EAF090359A
:102C5B0001E9F0903502E8F0D0F0227A007B007C9D
:102C6B0000601675F00A84AAF0600E75F00A84AB4A
:102C7B00F0600675F00A84ACF0EA2430FAEB2430ED
:102C8B00FBEC2430FC227A00900000790812339779
:102C9B00F4FB12337A122D6A123397B50313F41225
:102CAB00337A122D6AEA2408FAE5832420F583D9B6
:102CBB00DCBA2030900000123397FB9020001233C7
:102CCB0097B5031DF412337A122D6A90000012335C
:102CDB0097F4B503027A08EB90200012337A122D89
:102CEB006A022D59BA4067900000123397FB90206F
:102CFB0000123397B5032AF412337A122D6A90001F
:102D0B0000123397F4B5030F7A08EB9020001233BF
:102D1B007A122D6A022D59EB90200012337A122D64
:102D2B006A908000123397FB90A000123397B50383
:102D3B001DF412337A122D6A908000123397F4B57A
:102D4B0003027A28EB90A00012337A122D6A902599
:102D5B007FEAF022122C9190257FE0FAF599227CE4
:102D6B000075F032DCFED5F0FB227A80122DDB7B76
:102D7B0028902580122E1CF0A3DBF97AC0122DDBD4
:102D8B007B28122E1CF0A3DBF9227A80122DDB7B21
:102D9B0028902580E0FA122DFAA3DBF87AC0122DC9
:102DAB00DB7B28E0FA122DFAA3DBF8227A80122DB6
:102DBB00DB7400936007FA122DFAA380F4227AC019
:102DCB00122DDB7400936007FA122DFAA380F42204
:102DDB00C0F030111775F00075A0987802E230E75B
:102DEB000700D5F0F3022DF77800EAF2D0F022C0FD
:102DFB00F030111A75F00075A0987802E230E707F1
:102E0B0000D5F0F3022E1975A0987801EAF2D0F0F4
:102E1B0022C0F030111975F00075A0987802E230DD
:102E2B00E70700D5F0F3022E3A75A0987803E2D0AD
:102E3B00F02275A0807800EAF4F22275A080780267
:102E4B00EAF4F222AE82AF83902200EA23232325F9
:102E5B0082F58274003583F583E0F8A3E0F9EA2468
:102E6B004FF5A089F08E828F831233B2F2A308E85C
:102E7B00B5F003022EC3DBF1AE82AF83902200EAE2
:102E8B002323232582F58274003583F583E8BA006A
:102E9B000FC2ACF0200804D208D299D2AC022EBDDE
:102EAB00D20BF0902064EA14540F2582F582E0D205
:102EBB00E7F0E48E828F832274FF8E828F8322AEA3
:102ECB0082AF83902200EA2323232582F5827400AC
:102EDB003583F583E0F8A3E0F9EA244FF5A089F0F8
:102EEB008E828F831233B2B4F308DB1C0BA3E80280
:102EFB002F7DB4F408DB330BA3E8022F7DB4F56E02
:102F0B00DB4A0BA3E8022F7DA31233B2B4F3030207
:102F1B002F7914A3C082C08390250B2582F582E004
:102F2B00D083D082122FD3022F7DA31233B2B4F4ED
:102F3B0003022F7914A3C082C08390250B2582F541
:102F4B0082E0D083D082123024022F7DA31233B2C1
:102F5B00B4F503022F7914A3C082C08390250B25EF
:102F6B0082F582E0D083D082122FCF022F7D122FD9
:102F7B00CFA3B5F006022FC8022EEFDBFBAE82AF5C
:102F8B0083902200EA2323232582F5827400358364
:102F9B00F583E8BA000FC2ACF0200804D208D2992E
:102FAB00D2AC022FC2D20BF0902064EA14540F253E
:102FBB0082F582E0D2E7F0E48E828F832274FF8E5B
:102FCB00828F8322F208E8227F017E20C394644023
:102FDB000C1F7E31C394644004C394640E2464BEFE
:102FEB002002800EC0E0EE122FCFB5F0030230238B
:102FFB00D0E07E31C3940A40030E80F81E240AC031
:10300B00E0BE3003EF700AEE122FCFB5F0030230A3
:10301B0023D0E02430122FCF227F017E30C3946463
:10302B00400C1F7E31C394644004C394640E24642B
:10303B00C0E0EE122FCFB5F003023071D0E07E313D
:10304B00C3940A40030E80F81E240AC0E0BE30056C
:10305B00EF60027E30EE122FCFB5F003023071D04D
:10306B00E02430122FCF22200B03023113900012D9
:10307B00123397F5F0A3123397F58385F082A3E50E
:10308B00822411F582E5833400F583AE82AF839001
:10309B00206475A0907A00C082C0838E828F8312C9
:1030AB00339754E0B4E007D083D0820230FBD08357
:1030BB00D082E030E73AC2E7F0EAC4032402F8C05A
:1030CB0082C0838E828F83123397B40A168FF0746B
:1030DB0065F27FD7C2AFDFFE7475F27F24DFFED2BD
:1030EB00AFAFF0D083D08274A5F20808087406F253
:1030FB00A3C082C0838E828F83A3AE82AF83D08323
:10310B00D0820ABA1091C20B228D828E83A3A31296
:10311B0033B214540FC40375A0902402F8A31233D6
:10312B00B2F9C2AF7465F274A5F27FDEE9DFFED9A6
:10313B00FCF97475F27F6FDFFED9FC74B5F2D2AF78
:10314B002290000A1233976016758C00758A00D294
:10315B00A9D2AA7530FFF534853433D2078039C232
:10316B0007900009123397B4000875366A75350855
:10317B00801CB401087536877535E98011B40308D6
:10318B007536707535088006753688753508853641
:10319B008C85358AC2AAD2A9D20222E54E700302CF
:1031AB003248854E4F7A007B007800792A7D007576
:1031BB00F02675452075440085458285448312139E
:1031CB00A8AE82AF8374052582F58274003583F532
:1031DB00837C04C204C205123397A36002D204128B
:1031EB003397A3B4FF028002D205DCEB30041788BF
:1031FB00828983EEF0A3EFF0A3E54EC3954FF0A3C6
:10320B00A3A882A9830B3005198D8285F083EEF07C
:10321B00A3EFF0A3E54EC3954FF0A3A3AD82858337
:10322B00F00A854582854483A3A385824585834423
:10323B00D54F8590257EEBF090257DEAF022C2A834
:10324B0078087A007B10900012123397F5F0A312D6
:10325B003397F58385F082A3123397F523A3AE82C0
:10326B00AF83E5822410F582E5833400F5831233B6
:10327B0097FD75A021BD00067400D2E78055BD05F2
:10328B00067402D2E7804CBD06067402D2E7804377
:10329B00BD0C067401D2E7803ABDE0067404D2E798
:1032AB008031BD0D067405D2E78028BD1106740967
:1032BB00D2E7801FBD0E067407C2E78016BD0F064E
:1032CB007406D2E7800DBD10067408D2E780047433
:1032DB0003C2E7F2FCE82402F975A022ECF3BDE08F
:1032EB000302335C75A090EA2400F909097410F30A
:1032FB0019197402A21EB392E0BD00028003BD0E29
:10330B000444188011A21BB392E4A21C92E2A21DEA
:10331B005004C2E4D2E3F37407301F02740FF3EAD4
:10332B002401F9903372E5235407FC93F3EA240448
:10333B00F97488BC06028008BD05028003BD060235
:10334B007408F3EA2402F97401F3EA2405F974040E
:10335B00F38F838E82E82408F8EA2408FADB0280D4
:10336B0003023263D2A82244668899BBCCCCBBC083
:10337B0083C0E0E583C40354075390F84290E58380
:10338B00541F44C0F583D0E0F0D08322C083E58383
:10339B00C4035407C2AF5390F8429053831F438327
:1033AB00C0E0D2AFD08322300D04E493801E300AEC
:1033BB0003E08018C083E583C40354075390F8429D
:1033CB0090E583541F44C0F583E0D0832230070679
:1033DB00753000C28C32C0D0C0E0C083C08275D0C3
:1033EB001030071C758C00758A00D28CE40530B543
:1033FB0030037530FFD533058534338003023646F1
:10340B00D55003755010E538B40004C2B4800415D0
:10341B0038D2B4E537B40004C2B580041537D2B541
:10342B00300005D54102C200E528700302352A3071
:10343B00401B902001E014F07013C240B22090208A
:10344B0040E030E008902000E0A3F0D24030411B78
:10345B00902003E014F07013C241B221902040E0A1
:10346B0030E108902002E0A3F0D24130421B9020C3
:10347B0005E014F07013C242B222902040E030E21B
:10348B0008902004E0A3F0D24230431B902007E0C9
:10349B0014F07013C243B223902040E030E3089045
:1034AB002006E0A3F0D24330441B902009E014F037
:1034BB007013C244B224902040E030E408902008FE
:1034CB00E0A3F0D24430451B90200BE014F07013B6
:1034DB00C245B225902040E030E50890200AE0A3D9
:1034EB00F0D24530461B90200DE014F07013C2460D
:1034FB00B226902040E030E60890200CE0A3F0D2FA
:10350B004630472290200FE014F0701AC247B227C2
:10351B00902040E030E70F90200EE0A3F0D247E57B
:10352B0029700302362130481B902011E014F070F3
:10353B0013C248B228902041E030E008902010E000
:10354B00A3F0D24830491B902013E014F07013C243
:10355B0049B229902041E030E108902012E0A3F01D
:10356B00D249304A1B902015E014F07013C24AB2B6
:10357B002A902041E030E208902014E0A3F0D24AD8
:10358B00304B1B902017E014F07013C24BB22B90F2
:10359B002041E030E308902016E0A3F0D24B304CF2
:1035AB001B902019E014F07013C24CB22C902041E8
:1035BB00E030E408902018E0A3F0D24C304D1B9083
:1035CB00201BE014F07013C24DB22D902041E0305F
:1035DB00E50890201AE0A3F0D24D304E1B90201D31
:1035EB00E014F07013C24EB22E902041E030E6088A
:1035FB0090201CE0A3F0D24E304F1B90201FE01404
:10360B00F07013C24FB22F902041E030E7089020AA
:10361B001EE0A3F0D24F30020FD201853E83853FCF
:10362B0082A385833E85823F200710C28CE58A25C5
:10363B0035F58AE58C3536F58CD28CD082D083D09B
:10364B00E0D0D032C0D0C0E0C083C082C01F75D0E4
:10365B0018209811309903023723D01FD082D083C2
:10366B00D0E0D0D032C298E5874440F587309F2A0E
:10367B00C29F902100E0547FB400117401F0E587E4
:10368B0054BFF587759840D29C0236A57400F0E5BF
:10369B008754BFF5877598C0D29CE58754BFF587D3
:1036AB00902100E0547FB400030236CCA3E0F582F6
:1036BB0075833EE599F00582E582902101F0023792
:1036CB0020902101E0F8A3E0F9A3E0FAA3E0FBE5E9
:1036DB0099FF309A1030E70DC29A7B01E8FA0AEA9B
:1036EB006970027B00EB602175833E8A82EFF005E7
:1036FB0082E5826970047B00800FAA820B309A09E5
:10370B008882EB14F0EAF87B00902101E8F0A3A388
:10371B00EAF0A3EBF002365CC29910140302372DCA
:10372B00C15C902200E0F8A3E0B5180CE4902203F2
:10373B00F0A3F0C20802365CF8902100E0547FB48D
:10374B000031E8F8902204E0701275834F8882E014
:10375B00902203F0902201E004F08011F8902203F4
:10376B00E014B5180CE4902203F0A314F0D29B8064
:10377B0002C29B902201E075834FF582E0F599051B
:10378B0082E582902201F0A3A3A3E004F002365C51
:10379B00C0D0C0E0C0F0C083C08275D018753C109B
:1037AB00753D00753B00E53DB404004008B40F00C7
:1037BB0050030239D1E53B9090052582F582E0203C
:1037CB00E203023894C0E0902108E53B2582F582A4
:1037DB00E0FCA385823A858339547FB4000E909028
:1037EB0001E53B2582F582E0A2E5920C909003E582
:1037FB003B2582F582E0F5F0EC20E703023892548A
:10380B007FB40003023832853A82853983E0F58232
:10381B00E53D243FF583E5F0F00582E582853A82AC
:10382B00853983F0023892853A82853983E0FCA38F
:10383B00E0FDA3E0FEA3E0FFE5F0300C1030E70D58
:10384B00C20C7F01ECFE0EEE6D70027F00EF602567
:10385B008E82E53D243FF583E5F0F00582E5826D30
:10386B0070047F00800FAE820F300C098C82EF1436
:10387B00F0EEFC7F00902109E53B2582F582ECF010
:10388B00A3A3EEF0A3EFF0D0E020E0030239D19038
:10389B002208E53D2323232582F582E0FFA3E0B533
:1038AB001F22A3A37400F0A3F0909002E53B2582A6
:1038BB00F58274B8F0909005E53B2582F58274048F
:1038CB00F00239D1F5F085823A858339A3E0547F34
:1038DB00B400028008B4070280030239ADC0E0A334
:1038EB00E0FC600114FEA3E0FDD0E0B40705BC00D2
:1038FB00538003BC001FE5F0F582E53D2450F583B2
:10390B00E0FC0582E582853A82853983F0F5F0B5D6
:10391B001F070238ADEDB51E2B909002E53B2582BB
:10392B00F5827415F0909000E53B2582F582E0FE60
:10393B00A3A37415F0909000E53B2582F582EE442D
:10394B0004F08029909002E53B2582F5827415F0F6
:10395B00909000E53B2582F582E0FEA3A37415F061
:10396B00909000E53B2582F582EE54FBF0E5F0F5F7
:10397B0082E53D2450F583E0FE0582E582853A829F
:10398B00853983F00DECB51D047C007D00A3A3EC01
:10399B00F0A3EDF0909003E53B2582F582EEF0026B
:1039AB0039D1E5F0F582E53D2450F583E0F5F005DE
:1039BB0082E582853A82853983F0909003E53B2539
:1039CB0082F582E5F0F0053DE53B2408F53BD53C5F
:1039DB000280030237B1D082D083D0F0D0E0D0D0B8
:1039EB0032160016001459145F1465146B147115FC
:1039FB000715071507150A15101477148314B91436
:103A0B00BF14C514D714AD148F1495149B14A7149D
:103A1B00A114DD14E314E914EF15011507150715AF
:103A2B000715D615DC1516151C15E815EE14B31471
:103A3B008915221528152E1534153A1540154615DE
:103A4B00701576157C15821588158E1594159A159B
:103A5B00A015CA15D015E214FB15F41EDF1FCB20E1
:103A6B004E14F51600147D14CB14D1154C155215AC
:103A7B0058155E1564156A15A615AC15B215B81553
:103A8B00BE15C415071507150715071507150715D7
:103A9B00071507150715071507150715071507153B
:103AAB000715FA1507160016001600160016001655
:103ABB00000A56342B2056362E35330D0020563443
:103ACB002B2076362E35332020202020200020413D
:103ADB006C636F726E204D634272696465200020C7
:103AEB0053686F7720646174613A206261642000CF
:103AFB002053686F7720646174613A20206F6B20CC
:103B0B000020466C61672042616E6B2023203120C0
:103B1B002020466C61672042616E6B20232032208F
:103B2B002020466C61672042616E6B20232033207E
:103B3B002020466C61672042616E6B20232034206D
:103B4B00205374617465205661726961626C6520E3
:103B5B002357616974696E6720666F72202020207D
:103B6B00202020202020202020202020202020204A
:103B7B002020202020202020200065787465726E84
:103B8B00616C2073796E632E2E2E20202020202036
:103B9B00202020202020202020202020202020201A
:103BAB0020200045787465726E616C2073796E63AA
:103BBB0020202020202020202020202020202020FA
:103BCB002020202020202020202020007265636FE1
:103BDB0076657265642E2020202020202020202056
:103BEB0020202020202020202020202020202020CA
:053BFB00202020200045
:00000001FF
